:2000000002083312084EEF70FA22FF020DF37F20120EE6AE32AF33120396AF53120EE67F26
:200020002E120EE612036E22534554555020202100546D70443A00546D70433A004368727B
:200040006720454E440043687267202D45004368617267696E670045525220426174740075
:20006000436867642045525200436861726765645500436861726765645400446973636811
:200080006172670050623A20004274793A50622020004274793A4E694D6800453A2054698E
:2000A0006D657200453A64502F552F5400645073656E3A00542000AD07BD01087B43852F2E
:2000C00049852E48BD02087B44853149853048BD03087B45852949852A48AF03120EE67EAE
:2000E000007FB47C01120F16AF4912032B7F3A120EE6AF4812032B22C203E4F53F7E007FEF
:20010000287C01120F1612033B120003120F557540010202337433653E7002C2B4743265FE
:200120003E7002C2B37431653E7002C2B220B41405407D05AF40D3EF9D4003754001E4F59D
:200140003F02021574026540704220B31805297D17AF29D3EF9D400AE4F529E52A70037553
:200160002A05E4F53F30B2030202157405252AF52A7D37AF2AD3EF9D400CE5297005752AF9
:20018000058003E4F52AE4F53F020215A2B3E433FDA2B2E433FF5DFF60030202157401651E
:2001A000407008B205E4F53F02021574036540701305377D09AF37D3EF9D4003753701E425
:2001C000F53F8051740465407022B20720070CA206E433FF74FF2F9205800CA205E433FF3F
:2001E00074FF2F9206D205E4F53F80297405654070237464253BF53BE4353AF53A7C5F7D3A
:20020000B4AE3AAF3BD3EF9DEE9C4006753A52753B08E4F53FE53E6009E4F53ED2B2D2B3AC
:20022000D2B4E53F7008AF401208E5120003053F120EBA7D28AF3FC3EF9D5003020115D25C
:2002400003221205C712042F753458853C32853D33E4F52BE4F52DE4F52C02032812084EC9
:20026000AD077453653E70047B018002E4FBED4BFF60031200F8E4F535120D3812042FEED3
:200280004F70047B018002E4FB7C077DEEAE3CAF3DC3EF9DEE9C50047D018002E4FD7C0070
:2002A000AF037E00EF4DFFEE4CFE4F6006753458020328120BEF12042FEE4F70047B0180BA
:2002C00002E4FB7C077DEEAE3CAF3DC3EF9DEE9C50047D018002E4FD7C00AF037E00EF4D83
:2002E000FFEE4CFE4F6005753458803C12096912042FEE4F70047B018002E4FB7C077DEE11
:20030000AE3CAF3DC3EF9DEE9C50047D018002E4FD7C00AF037E00EF4DFFEE4CFE4F600526
:20032000753458800312088902025D7E00120396AF50120EE6AF4F120EE6227F0D120EE64F
:200340007F0A120EE6227820740C6021F9900F5C7A007B01E493A330E003EA4BFAEB2BFBFC
:200360005007A60208D9E98004D9E9A60222AF52120EE6AF51120EE6AF50120EE6AF4F1282
:200380000EE6227822900F687A1DEA6008E493A3F6081A80F5228E838F82E4FB7C007D0AF0
:2003A000AE83AF82120CEE74302FFD7F4FEF2BF8A6050BE583458260057508018003E4F5FB
:2003C000087C007D0AAE83AF82120D588E838F82EE4F600478018002E4F8AD03E4FCFE7F92
:2003E00005C3ED9FEC64806306809E500479018002E4F9AD007C00AF087E00EF5DFDEE5C34
:20040000FCAF017E00ED5FFFEC5EFE4F600302039C800A7F4FEF2BF87F30A6070B7F05C3B4
:20042000EB9F40EF22D2B5D2B7120EF0C2B722D2B5D2B7120D381207888E438F44C2B712EF
:2004400007E8AE43AF441205BFAC06AD077E077FD0C3ED9FEC9E5031900CC2200703900641
:2004600061E4FBEB2BFD7F08EF2DF8AE83AF820FEF70010EA60608A6070B7F09C3EB9F402E
:20048000E2E4F543F5440205B31207888E838F82E4FBAD03AB050BED2DFD7F08EF2DF9EBC0
:2004A0002BFD7F08EF2DF88606088607A70609A7077F09C3EB9F40DA858318858219AC1603
:2004C000AD17AE14AF15D3EF9DEE9C40047B018002E4FBAC16AD17AE18AF19D3EF9DEE9CCB
:2004E00040047D018002E4FD7C00AF037E00EF5DFFEE5CFE4F6006851416851517AC16AD14
:2005000017AE14AF15C3EF9DEE9C50047B018002E4FBAC16AD17AE18AF19C3EF9DEE9C50F7
:20052000047D018002E4FD7C00AF037E00EF5DFFEE5CFE4F6006851416851517AE08AF0914
:20054000E50B2FFDE50A3EFCAE0CAF0DED2FFDEC3EFCAE0EAF0FED2FFBEC3EFAAE10AF116E
:20056000E5132FFDE5123EFCAE14AF15ED2FFDEC3EFCAE16AF17ED2FF9EC3EF87F02AC0271
:20058000EB8FF005F08005CCC313CC13D5F0F8FD7F02AE00E98FF005F08005CEC313CE13A6
:2005A000D5F0F8FF2DFFEE3CFEC313FEEF13FF8E438F44AE43AF441205BF8E3C8F3D227CC4
:2005C000007D06120DD522D2B5C2B7752313752488C2AFE4F589438901758CFF7E5A7F4A75
:2005E0008F8AD28CC293D2A9D2AF120EBA120EC4227E007F57AB07AA067801C209C208C2CD
:200600000B74446534700E7E007F7BAB07AA067801D208D209744B6534700E7E007F69AB11
:2006200007AA067801D209C20874546534700E7E007F72AB07AA067801D209C208744565F9
:2006400034700E7E007F60AB07AA067801D209C208744365347037D208C2097E007F4EAB79
:2006600007AA067801E4F5487D14AF35D3EF9D400C7E007F3DAB07AA0678018011E53560E9
:200680000A7E007F46AB07AA06780185354874016536701EAC00AD01AE02AF03120F16E5BA
:2006A000487003020782AF4874302FFF120EE60207827402653670087F011200B70207823D
:2006C0007403653670087F021200B702078274046536700B12000E7F56120EE60207827433
:2006E000056536701CAF2D12032B7F3A120EE6AF2C12032B7F3A120EE6AF2B12032B0207F6
:20070000827406653670087F031200B70207827407653670157E007F377C01120F16AF388A
:2007200012032B7FDF120EE680587408653670157E007F317C01120F16AF3912032B7FDF39
:20074000120EE6803D74096536700F12086CA207E433FFBF012C05368028740A653670059D
:20076000120CDF801D740B6536700B120CC7200711E4F536800C740C653670061207C3E441
:20078000F536053612033B22E4FCFDD296D295D297C295C296D296C296D296E4FBC296D28C
:2007A00096ED2DFDEC33FCA297E433FFBF01050DED70010C0B7F0CC3EB9F40E1D295AE04C9
:2007C000AF05227E007F847C01120F16AE3AAF3B120396AF53120EE67F2E120EE6AF5212C3
:2007E0000EE6AF51120EE622C204C291120EBAC2AFD291E4F538800205383091FBD2AFC247
:2008000090120EBAC2AFD290E4F539800205393090FBD2AFAF3874FB2FFF12091A8F38AF5E
:200820003912091A8F39D20422C2B7C2B5120EF0D2B522E5A8C2AF5490758153A881760017
:2008400018B81FFAC0E0120EDFD0A8020242A2B3E433FDA2B2E433FF5DFDA2B4E433FF5D5C
:20086000FF70047D018002E4FDAF0522A205E433FFBF010B7E007F9B7C01120F1680097E73
:20088000007FA47C01120F1622E4F53575344BA200E433FFBF0103753454A201E433FFBF6D
:2008A0000103753445E4F52BE4F52DE4F52CE4F53F12042F80287E007F02120829E4F540D7
:2008C000120EBA05407D50AF40C3EF9D40F212042FEE4F7003753F01853C32853D33E53F06
:2008E00060D4AF3F228F4174016541700312086C7402654170057F031200B7740365417067
:2009000003120CDF740465417003120CC77405654170031207C312033B22AD077B1E7F981D
:20092000D3ED9F40027B287FA2D3ED9F40027B327FA7D3ED9F40027B3C7FACD3ED9F4002BA
:200940007B467FB1D3ED9F40027B507FB8D3ED9F40027B5A7FBFD3ED9F40027B647FC7D3B6
:20096000ED9F40027B6EAF0322753443E4F52BE4F52DE4F52CE4F535753F0075400AAF2998
:20098000E4FEFC7D3C120DD57C007D3C120DD5AA06AB07AF2AE4FEFC7D3C120DD5EF2BFFC4
:2009A000EE3AFE8E278F28C200C20112042F8E328F33853241853342020BE2852C2E852DE7
:2009C0002F7C017DF4AE3FAF40D3EF9DEE9C4006753F017540F475430A7D28AF38D3EF9DE4
:2009E0004015AF3874D82FFD7F0AED8FF084FD7F0AC3EF9DFF8F437C007D0AAE3FAF401233
:200A00000D58AA06AB07AF43AD077C00AE02AF03120DD5120829AF43AB07E4FAFC7D0AAEA1
:200A20003FAF40120D58AC06AD07AE02AF03120DD57C017DF4C3ED9FFFEC9EFE120EF0126F
:200A40000EBA7E007F0A120425120EBA12042F8E328F337C5F7DDCAE32AF33C3EF9DEE9C1C
:200A6000400479018002E4F97C077DEEAE32AF33D3EF9DEE9C50047D018002E4FDE532452F
:200A80003370047B018002E4FB7C00AF017E00EF4DFDEE4CFCAF037E00ED4FFFEC4EFE4FC7
:200AA0006008753518D201020BE274052540F540E4353FF53FA207E433FFBF01047901802E
:200AC00002E4F920050478018002E4F8AC32AD33AE3AAF3BC3EF9DFDEE9CFC7E007F0AC30B
:200AE000ED9FEC9E50047B018002E4FBAD007C00AF017E00EF5DFDEE5CFCAF037E00ED5F4D
:200B0000FFEC5EFE4F60037535197D14AF35C3E50795054003020BE2AC41AD42AE32AF338B
:200B2000C3EF9DEE9C40047B018002E4FBA207E433FFBF01047D018002E4FD7C00AF037EAB
:200B400000EF4DFFEE4CFE4F6011853241853342E4F535E4F525F526020BCB300503020B2C
:200B6000CB7D06AF37EF8DF0A4FFAD077C00AA32AB33AE41AF42C3EF9BFFEE9AFE120D581F
:200B80008F357C007DB4AE25AF26D3EF9DEE9C403AE4F525F5267B017D03AF37D3EF9D403F
:200BA000117D01AF37D3EF9D40047D018002E4FDAB05AF03E4FEFC7D06120DD5AC41AD42A9
:200BC000C3ED9FFFEC9EFE8E418F427D05AF35D3EF9D4003753518E5274528700575351726
:200BE000D2007D14AF35C3EF9D50030209BB22E4F535753444E4F52BE4F52DE4F52CE4F541
:200C00003FA207E433FFBF010875404C754190800675402675414812042F020CBD852C3077
:200C2000852D31120F5512042FE53C453D7003753F01AC40AD41AE3CAF3DD3EF9DEE9C5062
:200C40000479018002E4F97C5F7DDCAE3CAF3DC3EF9DEE9C40047D018002E4FD20B4047B5C
:200C6000018002E4FB7C00AF017E00EF4DFDEE4CFCAF037E00ED4FFFEC4EFE4F6005753FEE
:200C800001803475425A7D28AF39D3EF9D400EAF3974D82FFDAF42C3EF9DFF8F42AF427E75
:200CA00000120425AF42AD07E4FCFE7F5AC3EF9DFFEE9CFE120EF0853C32853D33E53F703B
:200CC00003020C1DAF3F2220070B7E007F927C01120F1680097E007F897C01120F16227EFE
:200CE000007FAD7C01120F16AF3712032B22120D58AE04AF0522752205E52270FC22C8A62E
:200D00000408A60508A60608A607C822C88604088605088606088607C822EC70078F828ECF
:200D200083E0FF22D5E0078F828E8393FF22D5E006C88F008607C822754809120CF6D5481D
:200D4000FAA204E433FDA202E433FF5DFF60083003031205F1C20222C000C001C002C00337
:200D6000C083C082AA04AB05A806A90775F000EA4B7006E4FEFF020DC805F0EA5480701730
:200D8000EB2BF582EA33F583D3E58299E583985006AA83AB8280E2E4F583F582E58225826B
:200DA000F582E58333F583C3E99BE89A4008C3E99BF9E89AF8A3EAC313FAEB13FBD5F0DCE7
:200DC000AE83AF82AC00AD01D082D083D003D002D001D00022C000C001ED8FF0A4F9A8F028
:200DE000ED8EF0A428F8EC8FF0A428FEAF01D001D00022C005C006C007C0E0C0D053D0E790
:200E0000C28C758CFF7E5A7F4A8F8AD28CE52260021522E5234524703A75231375248805E0
:200E20002B743C652B7005052CE4F52B743C652C7005052DE4F52CD2020526E5267002052F
:200E400025E52745286008E528152870021527B20A8008E524152470021523A208E433FDA6
:200E6000A209E433FF4DFF701AA20AE433FF74FF2F9293200A047D018002E4FD74FF2D9211
:200E800094801FA20AE433FDA208E433FFED5FFF74FF2F9293A209E433FFED5FFF74FF2FDF
:200EA0009294A298E433FFBF010585993EC298D0D0D0E0D007D006D00532754509120D3823
:200EC000D545FA22759840438920758DE8D28ED29C22EF2BFFEE3AFEED39FDEC38FC221213
:200EE000038312034622C2998F993099FDC299228E448F45E4F546F547800B120D380547FA
:200F0000E54770020546AA44AB45AC46AD47C3ED9BEC9A40E622744A120CFEE4F54E801B6F
:200F2000AF4E7E00AB07AA06E4F9F8744A120D0C120ED2120D1A120EE6054EAF4E7E00AB6C
:200F400007AA06E4F9F8744A120D0C120ED2120D1AEF70CC22120EBA120EBA2200000001CD
:200F600001000000000000000000000000000004000000000000000000002000000200004A
:050F80005A3C000000D6
:00000001FF
